:020000040000FA
:040000006F303A28FB
:040004000034003490
:08000800A000030EA100831209
:1000100005191128831601178312B2308100B1012E
:100020002C2883160113831203140B190310A80D37
:10003000A90DAA0DAB0DAC0DAC16FF302C02031DA3
:100040002C28FA302B02031D2C2832152A08AF0069
:100050002908AE002808AD008B100B11210E83007B
:06006000A00E200E0900B5
:0C007400203084008001840A80300402E7
:10008000031C3C28652183160C30850587018312EB
:10009000850187010730990000309A0010308316DF
:1000A0008E008312603083168F0083120030831617
:1000B00091009F008312C830831681008312313073
:1000C0009000003083168C00831210308B00A32127
:1000D00081018E018F010B118B100B108C018B177E
:1000E000802032198C204721B40B7E2803108519FB
:1000F0000314BA0DF0303A020319ED20A421702840
:1001000064003310B10A311F8B28AC01AB01AA0186
:10011000A901A801B101080032110130B7008B1309
:100120002030370783169B001C141A088312A40082
:100130001030370783169B001C141A088312A30083
:10014000A6000230A6060030370783169B001C1459
:100150001A088312A200A7000130A7068B17331CD0
:10016000B72822090339A200A309A409A509240874
:100170002F02031DE72823082E02031DE72822086B
:100180002D02031DE72801303702031DCC283E183D
:10019000CC283E143F14802102303702031DD5289D
:1001A000BE18D528BE143F14892103303702031D21
:1001B000DE283E19DE283E153F1492210430370216
:1001C000031DE728BE19E728BE153F149B21B70A77
:1001D00005303702031808008F280130B600B4003C
:1001E000B500B70085018701B2138020B40B09293F
:1001F000031085190314BA0DF0303A02031931299E
:10020000B51F8501B51F8701B50B09299630B500CB
:100210003B21321DF5283211331C13292D090339D6
:10022000AD00AE09AF092F1CF5282D0830020319C7
:10023000F5282D08B0002E1EF5288B132030370727
:10024000BC002F08BB00502110303707BC002E081F
:10025000BB00502100303707BC002D08BB005021E7
:100260008B1785018701B70AB60105303702031CD9
:10027000F528A32108003708B6080319B6000319AA
:1002800008001130850013308700B60308003F1CBA
:1002900008003F101030BC003E08BB005021080091
:1002A0008B133B0883161C159A0083123C08831697
:1002B0009B0055309D00AA309D009C1464009C1842
:1002C0005E291C1183128B170800831610309B00C7
:1002D0001C141A088312BE00831620309B001C14C5
:1002E0001A088312C2000130C21BC200C2080319DF
:1002F000C2000130D500D200EE30D000D10008009D
:100300000130D500D200EE30D000D1000130BE0067
:1003100008000130D500D200EE30D000D10002300C
:10032000BE0008000130D500D200EE30D000D10070
:100330000430BE0008000130D500D200EE30D000FD
:10034000D100BE01080008008F08031908008F01C2
:10035000C10B08004208C100D50B08005608D500A3
:1003600007303E050319DB29D21BD00AD21FD00368
:100370000A305002031CD629D0010930D21FD00008
:100380005203D2007F39031DD629D10A1030510201
:10039000031CCB29D1015022D2006022D40070224C
:1003A000D600D500D0010930D21FD000002385002F
:0C03B00024238700080085018701080055
:1004A00002308A0051083E1C572A883E8200BE1C3A
:1004B0005B2A883E82003E1D5F2A983E82000034FF
:1004C00002308A0051083E1C672AA83E8200BE1CEA
:1004D0006B2AB83E82003E1D6F2AB83E820000346F
:1004E00002308A0051083E1C772AC83E8200BE1C9A
:1004F0007B2AD83E82003E1D7F2AE83E82000134DE
:100510000734873407348734033483340334833413
:100520000B3403340F3407340B34033403340734EF
:10053000053487340734253483340334073489344D
:100540000B3403348F3405348B34113403340334C7
:1005500001340134023402340434043408340834DD
:10056000103410342034203440344034803480340B
:10057000083404340234803440348034103402347B
:10058000043410342034013404344034843480344E
:10059000093409340A340A34083408340834083475
:1005A0000834183408341834083418341034083433
:1005B000093429340A341A34283408340834083405
:1005C0000A34383408341A3408345834103448346F
:1005D000293409340A340A342834083408344834B5
:1005E0002834183488341834283418341034083433
:1006000003308A005008541C072B4B3E8200D41C38
:100610000B2B563E8200541D0F2B613E8200D41DD1
:10062000132B6C3E8200541E172B773E8200D41E83
:100630001B2B823E8200541F1F2B8D3E8200D41F35
:10064000232B983E8200003403308A005008541C4B
:100650002B2BA33E8200D41C2F2BAE3E8200541DB8
:10066000332BB93E8200D41D372BC43E8200541E6A
:100670003B2BCF3E8200D41E3F2BDA3E8200541F1C
:10068000432BE53E8200D41F472BF03E820000340E
:0A0696001034203401340234003423
:0A06A000003400340034003400344C
:0406AC0010343034A2
:1006B0003134333433343334333433343334333404
:0E06C2000034003400340034003400340234BC
:0606D0000334233433342F
:0806D800103420340134023417
:0C06E000003410342034013402340034A3
:0206EE001034C6
:1006F0002034013402340034003402340134203414
:020700001034B3
:0C070400103430343134333433343334A7
:080710003134303410340034A0
:06071A00333423340334E4
:0E072000023400340034023403342334333402
:10073000333400343334003433340034333400344D
:04074000333400341A
:0A07460000340034003400340234A3
:0A075000043401342034103408345E
:04075C000034003431
:1007600000340034023406340734273437343F343D
:0E07720008341834383439343D343F343F34C1
:060780003F343F343F341A
:08078800043401342034103464
:0C0790000A3404340134203410340A34DC
:02079E0008341D
:1007A000103420340134063406340134203410343B
:0207B00008340B
:0C07B40008341834383439343F343934F8
:0807C000383418340834003409
:0607CA003F3437342734F0
:0E07D0000734063406340734273437343F34F8
:1007E0003F3400343F3400343F3400343F3400346D
:0407F0003F3400345E
:084000000C000300060009009A
:02400E00CC33B1
:10420000010078007A007C007E007B0079007F004E
:104210007D007A0078007E007C00FF00FF00FF0038
:104220000000F200F600FA00FE00F200F600FA00CC
:10423000FE00F200F600FA00FE00FF00FF00FF00A3
:10424000010005000500050005000900090009003E
:1042500009000D000D000D000D00FF00FF00FF0024
:10426000FF00FF00FF00FF00FF00FF00FF00FF0056
:10427000FF00FF00FF00FF00FF00FF00FF00FF0046
:10428000FF00FF00FF00FF00FF00FF00FF00FF0036
:10429000FF00FF00FF00FF00FF00FF00FF00FF0026
:1042A000FF00FF00FF00FF00FF00FF00FF00FF0016
:1042B000FF00FF00FF00FF00FF00FF00FF00FF0006
:1042C000FF00FF00FF00FF00FF00FF00FF00FF00F6
:1042D000FF00FF00FF00FF00FF00FF00FF00FF00E6
:1042E000FF00FF00FF00FF00FF00FF00FF00FF00D6
:1042F000FF00FF00FF00FF00FF00FF00FF00DD00E8
:00000001FF
